:100000000C945D060C94471D0C94201D0C948506E1
:100010000C9485060C94131F0C9485060C94E51E15
:100020000C94581F0C9485060C9485060C94850638
:100030000C9485060C9485060C9485060C94850614
:100040000C94D61C0C9485060C94941D0C946E1D77
:100050000C9485060C9485060C9485060C948506F4
:100060000C94C61D0C9485066803180172681880EC
:10007000234020034C69676874734F4E04034F4E4E
:10008000042020202020BE5004B03B805F50046834
:100090003B0205680576380A01285004683B282F82
:1000A0006805183802004F680576380A00295004A0
:1000B000683B212650046832101E50046832111F1C
:1000C000C004BF1103696804800200EE8003680168
:1000D000EA1804FF0200E16804C00200AEC0036831
:1000E00001AA6818802340200350616E646F72611A
:1000F0002004032020042020202020F468188023DE
:10010000402003425420417564696F040320200499
:100110002020202020F36818802340200320415510
:100120005820492F5004032020042020202020E9BB
:1001300068188023402003555342617564696F0439
:10014000032020042020202020A1681880234020A4
:1001500003464D20626E64203104032020042020D9
:10016000202020C168188023402003414D20426E8A
:1001700064203204032020042020202020E5681879
:100180008023402003414D20426E6420310403202F
:1001900020042020202020E66818802340200346E9
:1001A0004D20426E642033040320200420202020B0
:1001B00020E368188023402003464D20626E6420AF
:1001C0003204032020042020202020C26805183893
:1001D00003004E68057638030020180A68390209C2
:1001E000003F000101776805183801004C0000004D
:1001F00000003E5B4F5B3E3E6B4F6B3E1C3E7C3EC9
:100200001C183C7E3C181C577D571C1C5E7F5E1CD6
:1002100000183C1800FFE7C3E7FF0018241800FF90
:10022000E7DBE7FF30483A060E2629792926407F8A
:10023000050507407F05253F5A3CE73C5A7F3E1C99
:100240001C08081C1C3E7F14227F22145F5F005F85
:100250005F06097F017F006689956A606060606063
:1002600094A2FFA29408047E040810207E201008A7
:10027000082A1C08081C2A08081E101010100C1E42
:100280000C1E0C30383E3830060E3E0E06000000C4
:10029000000000005F00000007000700147F147FCB
:1002A00014242A7F2A1223130864623649562050E8
:1002B0000008070300001C2241000041221C002A04
:1002C0001C7F1C2A08083E080800807030000808BF
:1002D000080808000060600020100804023E514930
:1002E000453E00427F400072494949462141494DFF
:1002F000331814127F1027454545393C4A49493186
:1003000041211109073649494936464949291E0004
:1003100000140000004034000000081422411414AE
:10032000141414004122140802015909063E415DCB
:10033000594E7C1211127C7F494949363E41414158
:10034000227F4141413E7F494949417F09090901D5
:100350003E414151737F0808087F00417F410020E2
:1003600040413F017F081422417F404040407F02CE
:100370001C027F7F0408107F3E4141413E7F0909F6
:1003800009063E4151215E7F0919294626494949FE
:100390003203017F01033F4040403F1F2040201FA8
:1003A0003F4038403F63140814630304780403613A
:1003B00059494D43007F414141020408102000414A
:1003C00041417F04020102044040404040000307D5
:1003D000080020545478407F28444438384444442A
:1003E00028384444287F385454541800087E0902A1
:1003F00018A4A49C787F0804047800447D40002061
:1004000040403D007F1028440000417F40007C04B4
:100410007804787C080404783844444438FC182470
:10042000241818242418FC7C080404084854545444
:100430002404043F44243C4040207C1C2040201CD9
:100440003C4030403C44281028444C9090907C44E0
:1004500064544C440008364100000077000000411D
:1004600036080002010204023C2623263C1EA1A1FC
:1004700061123A4040207A385454555921555579E3
:1004800041225454784221555478402054557940A3
:100490000C1E527212395555555939545454593904
:1004A000555454580000457C410002457D420001EE
:1004B000457C407D1211127DF0282528F07C545592
:1004C00045002054547C547C0A097F4932494949EB
:1004D000323A4444443A324A4848303A4141217A17
:1004E0003A42402078009DA0A07D3D4242423D3DE1
:1004F0004040403D3C24FF2424487E4943662B2F46
:10050000FC2F2BFF0929F620C0887E0903205454B4
:1005100079410000447D413048484A323840402209
:100520007A007A0A0A727D0D19317D2629292F2831
:10053000262929292630484D40203808080808086F
:10054000080808382F10C8ACBA2F102834FA000059
:100550007B000008142A142222142A14085500557E
:100560000055AA55AA55AAFF55FF55FF000000FFE8
:1005700000101010FF00141414FF001010FF00FFF3
:100580001010F010F0141414FC001414F700FF0005
:1005900000FF00FF1414F404FC141417101F1010B3
:1005A0001F101F1414141F00101010F00000000082
:1005B0001F101010101F10101010F010000000FF7E
:1005C000101010101010101010FF10000000FF1479
:1005D0000000FF00FF00001F10170000FC04F414CF
:1005E000141710171414F404F40000FF00F7141487
:1005F0001414141414F700F7141414171410101F03
:10060000101F141414F4141010F010F000001F1038
:100610001F0000001F14000000FC140000F010F088
:100620001010FF10FF141414FF141010101F0000FE
:100630000000F010FFFFFFFFFFF0F0F0F0F0FFFF11
:10064000FF0000000000FFFF0F0F0F0F0F384444A2
:100650003844FC4A4A4A347E02020606027E027E82
:100660000263554941633844443C04407E201E20C7
:1006700006027E020299A5E7A5991C2A492A1C4C6C
:100680007201724C304A4D4D303048784830BC626F
:100690005A463D3E494949007E0101017E2A2A2AE7
:1006A0002A2A44445F444440514A444040444A5109
:1006B000400000FF0103E080FF000008086B6B08AA
:1006C0003612362436060F090F06000018180000EF
:1006D000001010003040FF0101001F01011E001931
:1006E0001D1712003C3C3C3C0000000000000103D0
:1006F000070F1F3F7F0080C0E0F0F8FCFEDB40A446
:10070000A62EAF2000A1C8D300408DAED580A80092
:100710000060000000000000000000000000000079
:10072000E00000000000000000000000000001E008
:100730000000000000000000000000000001F000C8
:1007400000000000000000000000000003F00000B6
:10075000000000000000000000000007F0000000A2
:100760000000000000000000000007F8000000008A
:100770000000000000000000000FF800000003C0AF
:10078000007E000001E0007F0FF800000003C000C1
:10079000FE000001E000FFEFF800000003C000FED3
:1007A000000001E000FFFFF800000003C000F000BF
:1007B00000000F007FFE7FC0000003C000F00000BB
:1007C000000F003FFE7FF83FF1FBCFFCFEF3BC3D86
:1007D000EFE01FFE7FFF7FFBFFDFFEFEFFBC3DEF74
:1007E000E01FC6FFFF7FFBFFDFFEFEFFBC3DEFE02B
:1007F0000FE3C7FE787BC3DE1EF0FFBC3DEF0007B2
:10080000FF87FC787BC3DE1EF0F83C3DEF0001FF64
:10081000FFF0007BC3C01EF0F03C3DEF0001F37F12
:10082000E03FFBC3CFFEF0F03C3DEF0003E33F8031
:100830007FFBC3DFFEF0F03C3DEF0007E73C0078B4
:100840007BC3DE1EF0F03C3DEF0007FFBE00787B6F
:10085000C3DE1EF0F03C3DEF0007FFFE00787BC3D7
:10086000DE1EF0F03C3DEF000FFFFE007FFBFFDFE0
:10087000FEF0F03FFDEFE00FFFFF007FFBFFDFFE2C
:10088000F0F03FFDEFE00FF9FF003E79F9CF9EF069
:10089000F01F3DE7E01FF1FF000000000000000036
:1008A000000000001F80FF007FFFFFFFFFFFFFFF32
:1008B000FFFFE01C007F007FFFFFFFFEB46D888D0F
:1008C00018E000001F007FFFFFFFFE95AD7DB577AC
:1008D000E000000F007FFFFFFFFEA5AD9D8D19E03A
:1008E000000006007FFFFFFFFEB5ADEDB57EE00026
:1008F0000000000001800000000000000000000374
:100900008000000000000000000007C000000000A0
:10091000000000000007C000000000000000000010
:100920000FC00000000000000000001FE0000000F9
:100930000000000000001FE00000000000000000B8
:10094000003FE00000000000000000003FF0000059
:10095000000000000000007FF00000000000000028
:100960001FF87FF0000000000000003FFE7FF00055
:100970000000000000003FFF7FF0000000000000CA
:10098000001FFFFBE0000000000000000FFFF9FF68
:10099000C00000000000000FFFF9FFF80000000099
:1009A000000007FFF1FFFF00000000000003FC73E0
:1009B000FFFF80000000000001FE3FFFFF800000FD
:1009C00000000000FF1E0FFF000000000000007F7D
:1009D000FE1FFC000000000000003FFFFFF80000C9
:1009E00000000000000FDFFFE0000000000000003A
:1009F0001F19FFC0000000000000003F3CFF000086
:100A00000000000000007E7CF800000000000000F4
:100A1000007FFE7C0000000000000000FFFFFC00E3
:100A200000000000000000FFFFFE000000000000CA
:100A30000000FFFFFE0000000000000001FFEFFECD
:100A40000000000000000001FFCFFE0000000000D9
:100A5000000003FF07FE0000000000000003FC0789
:100A6000FE0000000000000003F003FE0000000094
:100A7000000000018000FE000000000000000000F7
:100A8000007E000000000000000000003E000000AA
:100A9000000000000000000C0000000000000780C3
:100AA00000FC000003C0000000078001FC00000300
:100AB000C0000000078001FC000003C00000000728
:100AC0008001E00000001E000000078001E000003F
:100AD000001E007FE3F79FF9FDE7787BDFC0FFF79B
:100AE000FFBFFDFDFF787BDFC0FFF7FFBFFDFDFF10
:100AF000787BDFC0F0F787BC3DE1FF787BDE00F05C
:100B0000F787BC3DE1F0787BDE0000F787803DE1B0
:100B1000E0787BDE007FF7879FFDE1E0787BDE00F9
:100B2000FFF787BFFDE1E0787BDE00F0F787BC3D93
:100B3000E1E0787BDE00F0F787BC3DE1E0787BDE2A
:100B400000F0F787BC3DE1E0787BDE00FFF7FFBFF8
:100B5000FDE1E07FFBDFC0FFF7FFBFFDE1E07FFBD2
:100B6000DFC07CF3F39F3DE1E03E7BCFC00000009F
:100B70000000000000000000FFFFFFFFFFFFFFFF7D
:100B8000FFFFC0FFFFFFFFFD68DB111A31C0FFFF51
:100B9000FFFFFD2B5AFB6AEFC0FFFFFFFFFD4B5B22
:100BA0003B1A33C0FFFFFFFFFD6B5BDB6AFDC057E5
:100BB000616974696E6720666F7220492D42757392
:100BC0000053706565642F52504D206D6F6E6974CF
:100BD0006F72004149204D6F64756C6520313100A2
:100BE0005353443133303620616C6C6F63617469E8
:100BF0006F6E206661696C65640052504D3A20004A
:100C0000206B6D2F68004D65747269633A20002077
:100C10002041637475616C3A2000202053796E6323
:100C200020553A2000202053796E6320443A20005A
:100C300020204175746F3A204F4646005461726718
:100C400065743A2000204D50480053706565643A41
:100C500020006804BF0201D000000000240027002B
:100C60002A0000000000250028002B0000000008DA
:100C70000002010000030407000000000000000063
:100C80002200FF21000000002300260029000404A8
:100C90000404040404040202020202020303030324
:100CA0000303010204081020408001020408102000
:100CB0000102040810203B20072011241FBECFEFA3
:100CC000D8E0DEBFCDBF25E0A4EAB1E001C01D92AF
:100CD000A033B207E1F711E0A0E0B1E0ECE0F5E508
:100CE00002C005900D92A43AB107D9F716E0CCE501
:100CF000D6E004C02197FE010E943929CB35D107E7
:100D0000C9F70E9465210C94792A0C94000008957B
:100D1000833081F028F4813099F08230A9F0089571
:100D20008730A9F08830C9F08430B1F48091800018
:100D30008F7D03C0809180008F778093800008951D
:100D400084B58F7784BD089584B58F7DFBCF809166
:100D5000B0008F778093B00008958091B0008F7DB0
:100D6000F9CFCF93DF93282F30E0F901E459F34F07
:100D70008491F901EE55F34FD491F901E257F34F05
:100D8000C491CC23A1F081110E948806EC2FF0E0E1
:100D9000EE0FFF1FEC57F34FA591B491EC91ED23AB
:100DA00081E090E009F480E0DF91CF91089580E048
:100DB00090E0FACF1F93CF93DF93282F30E0F90113
:100DC000E459F34F8491F901EE55F34FD491F901B1
:100DD000E257F34FC491CC23A9F0162F81110E9442
:100DE0008806EC2FF0E0EE0FFF1FEE59F34FA591B0
:100DF000B4918FB7F894EC91111108C0D095DE230F
:100E0000DC938FBFDF91CF911F910895DE2BF8CF38
:100E1000CF93DF9390E0FC01EE55F34F249182577E
:100E2000934FFC0184918823C9F090E0880F991FAB
:100E3000FC01E85AF34FA591B491FC01EE59F34F30
:100E4000C591D49161110DC09FB7F8948C912095F4
:100E500082238C938881282328839FBFDF91CF91A1
:100E60000895623051F49FB7F8943C91822F809599
:100E700083238C93E8812E2BEFCF8FB7F894EC91DE
:100E80002E2B2C938FBFEACF3FB7F89480917B0233
:100E900090917C02A0917D02B0917E0226B5A89B24
:100EA00005C02F3F19F00196A11DB11D3FBFBA2FFC
:100EB000A92F982F8827BC01CD01620F711D811DBC
:100EC000911D42E0660F771F881F991F4A95D1F741
:100ED00008958F929F92AF92BF92CF92DF92EF923E
:100EE000FF924B015C010E9444076B017C010E9450
:100EF00044076C197D098E099F09683E734081057E
:100F00009105A8F321E0821A9108A108B10888EEA2
:100F1000C80E83E0D81EE11CF11C81149104A104C9
:100F2000B10429F7FF90EF90DF90CF90BF90AF9082
:100F30009F908F9008952FB7F894609177027091E9
:100F400078028091790290917A022FBF08950895D6
:100F5000089508950895EF92FF920F931F93CF93F2
:100F6000DF938C017B01D0E0C0E0F701EC0FFD1FA7
:100F70006491662361F0D801ED91FC910190F081BC
:100F8000E02DC8010995892B11F02196EECFCE01F5
:100F9000DF91CF911F910F91FF90EF900895AF9245
:100FA000BF92CF92DF92EF92FF920F931F93CF9356
:100FB000DF936C017B018B01040F151FEB015E01B8
:100FC000AE18BF08C017D10759F06991D601ED914D
:100FD000FC910190F081E02DC6010995892B79F7EC
:100FE000C501DF91CF911F910F91FF90EF90DF909E
:100FF000CF90BF90AF900895FC01538D448D252F65
:1010000030E0842F90E0821B930B541710F0CF96A2
:10101000089501970895FC01918D828D981761F0D4
:10102000A28DAE0FBF2FB11D5D968C91928D9F5FEB
:101030009F73928F90E008958FEF9FEF0895FC01CA
:10104000918D828D981731F0828DE80FF11D858D7D
:1010500090E008958FEF9FEF0895FC01918D228D10
:10106000892F90E0805C9F4F821B91098F73992795
:10107000089583E892E00E942D0821E0892B09F46D
:1010800020E0822F089580E090E0892B29F00E94D3
:10109000390881110C9400000895FC01A48DA80F5B
:1010A000B92FB11DA35ABF4F2C91848D90E00196AA
:1010B0008F739927848FA689B7892C93A089B189CA
:1010C0008C91837080648C93938D848D981306C06B
:1010D0000288F389E02D80818F7D80830895EF92CF
:1010E000FF920F931F93CF93DF93EC0181E0888FE2
:1010F0009B8D8C8D98131AC0E889F989808185FFB2
:1011000015C09FB7F894EE89FF896083E889F98953
:1011100080818370806480839FBF81E090E0DF9155
:10112000CF911F910F91FF90EF900895F62E0B8DA8
:1011300010E00F5F1F4F0F731127E02E8C8D8E1163
:101140000CC00FB607FCFACFE889F989808185FFCA
:10115000F5CFCE010E944D08F1CFEB8DEC0FFD2FA6
:10116000F11DE35AFF4FF0829FB7F8940B8FEA8985
:10117000FB8980818062CFCFCF93DF93EC01888D94
:101180008823B9F0AA89BB89E889F9898C9185FD02
:1011900003C0808186FD0DC00FB607FCF7CF8C9190
:1011A00085FFF2CF808185FFEDCFCE010E944D08F3
:1011B000E9CFDF91CF910895EF92FF920F931F93A4
:1011C000CF93DF93EC01EC80FD806E157F050CF072
:1011D00070C057FF04C0240F351F50E040E08E81DF
:1011E0009F81FA01E20FF31F8E179F071CF49C01E9
:1011F000241B350B121613060CF05BC0922F842FA4
:101200008695869586958E9DD0018F9DB00D112473
:101210006A0F7B1FAF8DB8A1A60FB71F477049F1AA
:1012200088E0841B482F682F70E0FB01EB50F94FDA
:10123000E491281708F063C0621B71092FEF30E0BA
:1012400002C0359527956A95E2F7E2230130110532
:1012500039F0B0F10230110561F58C91E82702C038
:101260008C91E82BEC93941720F12C813D81A20FF7
:10127000B31FE92FE41BE83078F00230110521F5A7
:101280008E2F9C9190959C932C813D81A20FB31F32
:1012900088508830B0F7E770EE2359F0F0E0E35162
:1012A000F94FE49101301105F9F010F10230110508
:1012B00019F1DF91CF911F910F91FF90EF90089559
:1012C000E0958C91E823CECF81E00115110509F45A
:1012D00080E081959E2F8C932C813D81A20FB31FBE
:1012E00098509830C0F7D7CF8C91E82BEC93E1CF92
:1012F000E0958C91E823FACF8C91E827F7CF013065
:10130000110509F4ADCFE0F20230110509F4A5CFC3
:10131000AE0DBF1DAECF0F931F93CF93DF9377FF1B
:1013200004C0260F371F70E060E0DC011496CD91F9
:10133000DC91FB01E20FF31FCE17DF071CF49E01C7
:10134000261B370B121613064CF5FA0157FD37967C
:10135000A3E0F595E795AA95E1F7EC9FD001ED9F05
:10136000B00DFC9FB00D11246A0F7B1FDC015F964E
:10137000ED91FC91E60FF71F4770552781E090E053
:1013800001C0880F4A95EAF7482F0130110559F03E
:10139000A8F02E0F3F1F02301105E1F0DF91CF9131
:1013A0001F910F9108952E0F3F1FE217F307B1F31E
:1013B0008191DF011197842B8C93F7CF80952E0FAD
:1013C0003F1FE217F30751F39191DF011197982323
:1013D0009C93F7CFE217F30709F38191DF0111978F
:1013E00084278C93F7CF0F931F93FA01DC01569655
:1013F0004C9156974230E9F04330A1F1413061F50C
:1014000014964D915C91DA01AE1BBF0BFD01E21BFE
:10141000F30B77FD0BC0DC0116964D915C916417C0
:10142000750724F4AB01BF010E948B091F910F9136
:10143000089514964D915C91DA01A61BB70BBD017E
:1014400061507109DC0116964D915C91DA01AE1B79
:10145000BF0BFD01E21BF30B77FDE8CFAF010E944C
:10146000DC08E4CF16964D915C91DA01A61BB70B10
:10147000BD0161507109CDCF0F931F93FA01DC01BB
:1014800056964C9156974230A9F0433091F1413035
:1014900019F514964D915C91DA01AE1BBF0BFD015D
:1014A0003197F7FD04C0AB01BF010E94DC081F911A
:1014B0000F91089514964D915C91DA01A61BB70B1C
:1014C000BD01DC0116964D915C91DA01AE1BBF0B9C
:1014D000FD013197621B730BF7FDE9CFDC01169616
:1014E0004D915C91E417F50714F7AF010E948B0949
:1014F000DECF16964D915C91DA01A61BB70BBD01AC
:10150000621B730BCECFFC0177FD64C08085918593
:10151000681779070CF05EC057FD5CC08285938523
:10152000481759070CF056C086898230B1F08330D5
:1015300029F1813041F484819581841B950BAB01A5
:10154000BC01615071092130310509F108F443C033
:101550002230310509F463C0089584819581DC014E
:10156000A61BB70BBD016150710986819781DC0113
:10157000A41BB50BAD0141505109E5CF8681978180
:10158000861B970BBA01AC0141505109DCCFCA014F
:1015900057FD0796A3E095958795AA95E1F7A48155
:1015A000B5818A9F90018B9F300D9A9F300D112439
:1015B000620F731F078CF0A1E02DE60FF71F477035
:1015C000552721E030E001C0220F4A95EAF78081DB
:1015D000822B80830895CA0157FD079633E09595C5
:1015E00087953A95E1F7A481B5818A9F90018B9FF9
:1015F000300D9A9F300D1124620F731F078CF0A1DC
:10160000E02DE60FF71F4770552781E090E001C0FD
:10161000880F4A95EAF7809590818923DACFCA012D
:1016200057FD079623E0959587952A95E1F7A481C4
:10163000B5818A9F90018B9F300D9A9F300D1124A8
:10164000620F731F078CF0A1E02DE60FF71F4770A4
:10165000552721E030E001C0220F4A95EAF780814A
:101660008227B7CF08958EBD00000DB407FEFDCFD1
:101670008EB508958CBD9DBD08950895FC016370DD
:10168000668B8481958126813781613039F06330A2
:1016900029F09187808733872287089531872087B3
:1016A0009387828708952F923F924F925F926F9215
:1016B0007F928F929F92AF92BF92CF92DF92EF92E2
:1016C000FF920F931F93CF93DF93CDB7DEB76A9747
:1016D0000FB6F894DEBF0FBECDBF9A8F898F7A8385
:1016E00069834A01D22E18870F833701BC2CDC0195
:1016F00059962D913C915A972115310509F015C144
:1017000018968D919C911997681779070CF0D7C19D
:101710001A968D919C91481759070CF0D0C14C2C0A
:10172000512CB6E0CB9E600D711D11247C876B8718
:10173000161617060CF0C3C1EA2DF0E0FA87E98708
:1017400093E0EE0FFF1F9A95E1F7F88BEF87CF013B
:10175000840F951F181619060CF0B1C1A98DBA8D0A
:1017600058968C91811104C0BFEABD1508F4D3943A
:10177000A98DBA8DED91FC9111970284F385E02D2E
:10178000CD010995B5E0DB9EC0011124E981FA8104
:10179000FC83EB83312C212C9C0123513E4F388F4D
:1017A0002F8B4A2D50E05E8B4D8BEF89F88DE20D2B
:1017B000F31D44919E828D82D12CC12C69817A8146
:1017C000620D731D7A8B698B842F90E09C8B8B8BC1
:1017D000E98DFA8DA081B18140FF82C0F1E0BF1296
:1017E0006FC0AF126DC01C96ED91FC912F813885B2
:1017F000A4014C0D5D1D69897A89898D9A8D0995A1
:10180000EB89FC89F595E7954E2F5FEFC51AD50A50
:101810006D817E818D899E89680F791F7E836D839E
:1018200098E0C916D10481F6AFEF2A1A3A0AEB8183
:10183000FC81E40DF51DFC83EB83F5E02F163104EC
:1018400009F0B3CF2F81388526153705B9F0A98D5A
:10185000BA8DED91FC91B1E0BB1257C0AB1255C0EF
:1018600069817A816B5F7F4F0088F189E02D830168
:1018700028E030E0A401898D9A8D0995A98DBA8D53
:10188000ED91FC9111970688F789E02DCD016A96BC
:101890000FB6F894DEBF0FBECDBFDF91CF911F9181
:1018A0000F91FF90EF90DF90CF90BF90AF909F90FF
:1018B0008F907F906F905F904F903F902F90099402
:1018C0001E96ED91FC91EF80F88409851A859201AE
:1018D0004D815E816B817C81898D9A8D099590CF38
:1018E0002F8138852615370509F48ACF31E0B312E8
:1018F00007C0A31205C01C96ED91FC91930178CF0F
:101900001E96ED91FC917301E0CF6B857C85641987
:1019100075090684F785E02D73010F8518899201FA
:10192000A401898D9A8D0995A9CFF90134969491D6
:10193000329745915491D91AB7E0DB9E400D511D65
:101940001124F901259134913C8B2B8BFA012590C0
:101950003490FA013296749031963491398B3296E4
:1019600064903196449041E04C1518F04A1508F007
:101970007FC0662D062C000C770B7C836B83842D37
:10198000042C000C990B9E838D83A98DBA8DED914B
:10199000FC9111970284F385E02DCD010995512C1E
:1019A000D12CC12CEA2DF0E0FA87E9872B2D30E00D
:1019B0003C872B87A401440D511D47FC5A95588F35
:1019C0004F8B69817A81660D711D67FC7A957E87E0
:1019D0006D877989C71608F051CF2C2D30E04D81E5
:1019E0005E81420F531FA985BA854A9FC0014B9F54
:1019F000900D5A9F900D1124FC01E80DF91DF88BF4
:101A0000EF87852D612C4F89588D420F531F5E8BB8
:101A10004D8B671408F050C044244394480E8770DF
:101A200041F4C1010196EB89FC89E20DF31DD490CC
:101A30001C01D7FE19C0A98DBA8DED91FC91662DC0
:101A400070E0B1E0BB1219C0AB1217C02D853E8506
:101A5000620F731F0484F585E02D2F8138854D8931
:101A60005E89898D9A8D0995DD0C6394842DD1CF83
:101A70001E821D821C821B8288CF4B815C81640F79
:101A8000751FAB85BC856A9FC0016B9F900D7A9FC7
:101A9000900D112469817A81680F791F0684F7857A
:101AA000E02DEF80F88409851A859D014F855889BE
:101AB000898D9A8D0995D8CF570CC3948ACF6A9691
:101AC0000FB6F894DEBF0FBECDBFDF91CF911F914F
:101AD0000F91FF90EF90DF90CF90BF90AF909F90CD
:101AE0008F907F906F905F904F903F902F900895D0
:101AF0008F929F92AF92CF92EF92FF920F931F938C
:101B0000CF93DF93EC01262F898D9A8D009709F0F2
:101B100051C06A30D1F41D861C868D8948E0849FAF
:101B2000900111248E859F85820F931F9F878E873A
:101B300081E090E0DF91CF911F910F91FF90EF90A6
:101B4000CF90AF909F908F9008956D3089F3CC889F
:101B5000AD888F898823C1F08C859D8536E0C39E32
:101B6000800D911D1124488559854817590764F443
:101B70004E855F851D861C8638E0A39EC00111241A
:101B8000840F951F9F878E87EA88FB8808891989AB
:101B90004E855F856C857D85CE010E94530B2C8917
:101BA0008C859D8546E0249F800D911D11249D8785
:101BB0008C87BECF6A3069F41D861C86FC0138967E
:101BC000E4912D898E859F85E29F800D911D1124C2
:101BD000ADCF6D3009F4ACCFFC013496349163176E
:101BE00008F4A6CF3296E491E61708F4A1CFFC01E1
:101BF000329685909490462F431B342F47E0349FB4
:101C0000800C911C1124F401329634913196E491A8
:101C10003323A9F1EE2399F1CC88F4013596E491B0
:101C2000AD884F89442301F10E2E000CFF0BE30F0A
:101C3000F11DCE9EA001CF9E500D11246C857D8597
:101C4000460F571F68857985641775076CF44E85B4
:101C50005F851D861C86FC013896E491AE9E400D82
:101C6000511D11245F874E87EA88FB8808891989EE
:101C70004E855F856C857D85CE010E94530BF401F6
:101C80003496E4912C898C859D85E29F800D911D71
:101C900011248DCF6F927F928F929F92AF92BF92BD
:101CA000CF92DF92EF92FF920F931F93CF93DF9328
:101CB000EC016B015A0139014801E881F981028484
:101CC000F385E02D0995E881F9810288F389E02DFB
:101CD00087019301A501B601CE010995A501480D23
:101CE000591D41505109E881F9810288F389E02D9D
:101CF0009301B601CE010995E881F9810088F18947
:101D0000E02D9401A501B601CE010995C60CD71CA2
:101D1000B60161507109E881F9810088F189E02DEF
:101D20009401A501CE010995E881F9810688F7891A
:101D3000E02DCE01DF91CF911F910F91FF90EF9099
:101D4000DF90CF90BF90AF909F908F907F906F90DB
:101D500009946F927F928F929F92AF92BF92CF928F
:101D6000DF92EF92FF920F931F93CF93DF935C016B
:101D7000EB016A01490138018701DC01ED91FC9119
:101D80006217730719F5641675062CF0962D872DCA
:101D90003A01C92ED82E9601261937092F5F3F4FD9
:101DA000048CF58DE02DA301BE01C5010995DF91DD
:101DB000CF911F910F91FF90EF90DF90CF90BF9048
:101DC000AF909F908F907F906F9008954615570524
:101DD00091F42617370724F0892D4B01C22FD82FF5
:101DE0009E01281939092F5F3F4F068CF78DE02D92
:101DF000A601B401DACF0284F385E02D0995D5015F
:101E0000ED91FC910488F589E02D83019401A601F0
:101E1000BE01C5010995D501ED91FC910688F789B0
:101E2000E02DC501DF91CF911F910F91FF90EF90B1
:101E3000DF90CF90BF90AF909F908F907F906F90EA
:101E40000994EF92FF920F931F93DC011A960D9164
:101E50001C911B9718962D913C911997ED91FC912F
:101E600000A0F1A1E02D7B0150E040E070E060E0D7
:101E700009951F910F91FF90EF9008954F925F92F7
:101E80006F927F928F929F92AF92BF92CF92DF928A
:101E9000EF92FF920F931F93CF93DF936C012B016F
:101EA0005A0139014801DC01ED91FC910284F3856E
:101EB000E02D0995E201640C751CD601ED91FC91B1
:101EC000C615D7055CF40088F189E02D87019401DF
:101ED000A501BE01C60109952196EFCF0688F789B5
:101EE000E02DC601DF91CF911F910F91FF90EF90F0
:101EF000DF90CF90BF90AF909F908F907F906F902A
:101F00005F904F9009948F929F92AF92BF92CF9221
:101F1000DF92EF92FF920F931F93CF93DF93EC0129
:101F20005B014A016901E881F9810284F385E02DB2
:101F3000099595012C0D3D1D21503109E881F9814C
:101F40000488F589E02D78018401A401B501CE0152
:101F50000995E881F9810688F789E02DCE01DF91A6
:101F6000CF911F910F91FF90EF90DF90CF90BF9096
:101F7000AF909F908F9009948F929F92AF92BF9253
:101F8000CF92DF92EF92FF920F931F93CF93DF9345
:101F9000EC015B014A0169017801E881F981028461
:101FA000F385E02D0995C80CD91C86010150110953
:101FB000E881F9810488F589E02D9501A401B50136
:101FC000CE010995E881F9810688F789E02DCE01D7
:101FD000DF91CF911F910F91FF90EF90DF90CF9005
:101FE000BF90AF909F908F900994EF92FF920F93C4
:101FF0001F93DC01ED91FC9100A0F1A1E02D09956A
:102000001F910F91FF90EF9008950F931F93DC01A4
:10201000ED91FC91068CF78DE02D09951F910F91A4
:1020200008950F931F93DC01ED91FC91048CF58DC5
:10203000E02D09951F910F910895DC01ED91FC9120
:102040000084F185E02D09943F924F925F926F9248
:102050007F928F929F92AF92BF92CF92DF92EF9238
:10206000FF920F931F93CF93DF935C017B014A0193
:102070006901390187E0680E711C93E075946794DB
:102080009A95E1F72B01400E511E10E000E0312C33
:10209000D0E0C0E0CE0187709927330C892B59F42A
:1020A000FE0183E0F595E7958A95E1F7E00FF11FD2
:1020B000E80DF91D349037FE0AC021E030E0A70199
:1020C000B5016C0F7D1F84ED94E00E941D102196D8
:1020D000CC16DD06F9F68FEFE81AF80A060D171D83
:1020E000E414F504A9F6DF91CF911F910F91FF90B1
:1020F000EF90DF90CF90BF90AF909F908F907F90A8
:102100006F905F904F903F9008952F923F924F9223
:102110005F926F927F928F929F92AF92BF92CF9277
:10212000DF92EF92FF920F931F93CF93DF9300D034
:1021300000D000D0CDB7DEB73C016A013E832D83CD
:10214000FC82EB825801A41AB50AB7FE03C0B19411
:10215000A194B1088D809E80861A970A97FE03C0CD
:102160009194819491088A149B045CF0902F812FA4
:102170000D811E819D838E839C2D8D2D6B01692F7A
:10218000782F0C151D055CF09D818E817E836D83FB
:10219000692F782F902F812F8601C92ED82E1601F6
:1021A000201A310A2B012D813E81421A530A57FE13
:1021B00003C0519441945108710137FE03C03FEFB1
:1021C000E31AF30AF594E7948D819E8186179707A9
:1021D0005CF5A1E0B0E0BA83A983C016D1064CF14A
:1021E000D301ED91FC910484F585E02D2B813C8198
:1021F000A8016D817E818A149B041CF04D815E8153
:10220000B801C3010995E418F508F7FE0AC02D814D
:102210003E8189819A81280F391F3E832D83E20CEC
:10222000F31C0F5F1F4FD9CF2FEF3FEF3A83298366
:10223000D4CF26960FB6F894DEBF0FBECDBFDF9188
:10224000CF911F910F91FF90EF90DF90CF90BF90B3
:10225000AF909F908F907F906F905F904F903F9046
:102260002F900895089520911102260F3327331FD0
:1022700021323105ECF420913502FC0190E080E040
:10228000243069F082E00895A09111022191AC01FF
:102290004F505E4FA40FB52FB11D2C93019686179A
:1022A00098F380911102680F6093110280E0089505
:1022B00081E008951092350281E0809337021092F8
:1022C000360261E082E10E94DA0661E083E10E9469
:1022D000DA06E9EBF0E080818E7F808380818D7F5C
:1022E000808388E48093B80085E48093BC000895DF
:1022F000CF93DF9391E09093F0018823B9F0C091E0
:10230000B800D091BA008091BC008A7B8093BC0059
:1023100060E082E10E94DA0660E083E10E94DA0672
:102320000E945A11D093BA00C093B800DF91CF91A8
:102330000895E091610280916002E81730F4F0E0C6
:10234000E553FE4F808190E008958FEF9FEF089551
:1023500090916102809160022FEF3FEF981748F44F
:10236000E92FF0E0E553FE4F208130E09F5F90932E
:102370006102C90108958091600290916102891BF8
:10238000990B0895CF92DF92EF92FF920F931F93D4
:10239000CF93DF937C01CB018A012091820222231B
:1023A00089F0EB016B01C40ED51ECC15DD0569F07B
:1023B0006991D701ED91FC910190F081E02DC70169
:1023C0000995F3CF642F0E943311C801DF91CF919B
:1023D0001F910F91FF90EF90DF90CF900895CF93D2
:1023E000DF931F92CDB7DEB769832091820222234B
:1023F000F9F020917F02203258F021E030E0FC011A
:102400003383228390E080E00F90DF91CF91089595
:1024100080918002E82FF0E0E555FE4F998190838E
:102420008F5F8093800280937F0281E090E0ECCF09
:1024300061E0CE0101960E943311F7CFCF92DF9277
:10244000EF92FF920F931F93CF93DF93D0917F0270
:1024500081E0D13208F09CC0C09181020E94440703
:102460006B017C018091350281116CC082E0809308
:10247000350281E0809337028FEF8093340210920F
:102480005902D0935802ABEAB1E0E8E3F2E080E011
:10249000D8138DC010925A0280915A02CC0FC82BCB
:1024A000C0935A0280913602813009F084C01092A4
:1024B00036020E9444076B017C0180915A0280938E
:1024C000BB008091EC019091ED01A091EE01B091E3
:1024D000EF01892B8A2B8B2BA1F00E9444070091DE
:1024E000EC011091ED012091EE013091EF016C199A
:1024F0007D098E099F09061717072807390708F471
:1025000042C08091BC0083FDD8CF85EC8093BC0095
:102510000E9444076B017C0180913502823009F4EE
:102520004CC0809134028F3F09F469C0809134021D
:10253000803209F466C080913402803309F463C0AC
:1025400084E026C08091EC019091ED01A091EE0114
:10255000B091EF01892B8A2B8B2B09F483CF0E943A
:1025600044070091EC011091ED012091EE013091B2
:10257000EF016C197D098E099F09061717072807B7
:10258000390708F06FCF8091EB010E94781185E048
:102590001092800210927F0210928202DF91CF91FE
:1025A0001F910F91FF90EF90DF90CF9008959D9134
:1025B00091938F5F6DCF85EEA9CF8091EC019091C3
:1025C000ED01A091EE01B091EF01892B8A2B8B2BAD
:1025D00009F4A2CF0E9444070091EC011091ED0193
:1025E0002091EE013091EF016C197D098E099F0950
:1025F000061717072807390708F08ECFC4CF80E0E9
:10260000C7CF82E0C5CF83E0C3CFEF92FF920F9395
:102610001F93CF93DF937C01C62F8091F10490919B
:10262000F204009709F459C02091F50431E0309389
:102630008202209381021092800210927F02DC01BC
:10264000ED91FC910190F081E02D60E0099587010A
:10265000EE24E394F12CD1E0C1508091F1049091EB
:10266000F204CF3F91F1B0E2EB16F104D8F00E94F2
:102670001E128091F1049091F2042091F504D09300
:102680008202209381021092800210927F02DC016C
:10269000ED91FC910190F081E02D60E00995EE2430
:1026A000E394F12C8091F1049091F204F80164918B
:1026B000DC01ED91FC910190F081E02D0995BFEFD7
:1026C000EB1AFB0A0F5F1F4FC7CFDF91CF911F910E
:1026D0000F91FF90EF900C941E12E0910105F09184
:1026E0000205908180910705809589238083870169
:1026F000C15008F438C0F80184912091EF04309162
:10270000F004232B29F00E94330B0F5F1F4FF0CFF3
:1027100028E030E040E8E091FD04F091FE04909163
:102720000505582F5423D9F05081952B9083E091C3
:10273000FF04F0910005908150910605952B908340
:10274000E091FF04F091000550819091060590956D
:1027500095239083469521503109E9F6D6CF5081D3
:1027600090959523E3CFDF91CF911F910F91FF902B
:10277000EF9008951F93CF93DF93EC018D8D9E8D85
:10278000009721F1162F29A131E030938202209386
:1027900081021092800210927F02DC01ED91FC9187
:1027A0000190F081E02D60E009958D8D9E8DDC011A
:1027B000ED91FC910190F081E02D612F09958D8DB7
:1027C0009E8DDF91CF911F910C941E12ADA5BEA5D9
:1027D0009C918BA9809589238C938B8D9C8D892BC3
:1027E00031F0862FDF91CF911F910C94330B28E0AD
:1027F00030E080E8A9A5BAA599A9462F4823C1F0E1
:102800004C91942B9C93ABA5BCA59C914AA9942B6D
:102810009C93ABA5BCA54C919AA9909594239C93AD
:1028200086952150310931F7DF91CF911F9108959D
:102830004C9190959423E6CFDF92EF92FF920F9305
:102840001F93CF93DF938091F1049091F204892B31
:1028500009F4A5C02091090530910A0540910B05A6
:1028600050910C0560E074E284EF90E00E9403292F
:1028700020513109410951095695479537952795BA
:102880002093B80064E080E89CE00E9405138091EA
:10289000D8049091D9048034910509F097C060E282
:1028A00084ED94E00E94BA136091D804615E84EDD7
:1028B00094E00E94BA132091DA043091DB04C9013C
:1028C000079697FD079633E0959587953A95E1F73A
:1028D0002091D8043091D904829F8001839F100DEC
:1028E000929F100D1124C091F304D091F4048091B3
:1028F000F1049091F2040C0F1D1F009709F498C089
:102900002091F50431E030938202209381021092ED
:10291000800210927F02DC01ED91FC910190F08128
:10292000E02D60E40995EE24E394F12CDD24D394AA
:102930008091F1049091F2040C171D0709F44FC027
:10294000B0E2EB16F104D8F00E941E128091F1045F
:102950009091F2042091F504D0928202209381029A
:102960001092800210927F02DC01ED91FC910190A7
:10297000F081E02D60E40995EE24E394F12C809140
:10298000F1049091F2046991DC01ED91FC910190C8
:10299000F081E02D0995BFEFEB1AFB0AC9CF8091BA
:1029A000EF049091F004892B31F080911205909101
:1029B00013050E943A0BE0910305F0910405908104
:1029C000809108058095892380835CCF60E084ED49
:1029D00094E00E94BA136091D804615068CF0E94BD
:1029E0001E128091F1049091F204892B09F461C0C8
:1029F00020910D0530910E0540910F055091100565
:102A000060E074E284EF90E00E94032920513109D4
:102A10004109510956954795379527952093B80058
:102A2000DF91CF911F910F91FF90EF90DF9008956C
:102A3000E0910105F0910205808190910705892BB5
:102A400080830C171D0769F289912091EF04309162
:102A5000F004232B19F00E94330BF3CF28E030E071
:102A600040E8E091FD04F091FE0490910505582F97
:102A70005423D9F05081952B9083E091FF04F0917D
:102A80000005908150910605952B9083E091FF04FD
:102A9000F0910005508190910605909595239083C3
:102AA000469521503109E9F6CCCF50819095952378
:102AB000E3CFE0910305F091040580819091080532
:102AC000892B8083ADCF1F93CF93DF93EC01162F1B
:102AD0008D8D9E8D892BB1F12DA93EA94FA958ADA1
:102AE00060E074E284EF90E00E94032920513109F4
:102AF0004109510956954795379527952093B80078
:102B000066EA111167EACE010E94BA138D8D9E8D7F
:102B1000892B41F129AD3AAD4BAD5CAD60E074E27B
:102B200084EF90E00E9403292051310941095109A5
:102B300056954795379527952093B800DF91CF910B
:102B40001F9108958B8D9C8D892B21F08EAD9FADAB
:102B50000E943A0BEFA5F8A990818CA98095892352
:102B60008083CECFEFA5F8A980819CA9892B808393
:102B7000E5CF90E080E00895FC0184819581228179
:102B800033812817390771F0860F971F6081718193
:102B90000E9425290680F781E02DE80FF91F80812A
:102BA00090E008958FEF9FEF0895FC018481958157
:102BB000228133812817390741F0860F971F6081E2
:102BC00071810E942529958384830895FC01462FF5
:102BD00022813381C9010196608171810E9425297A
:102BE000648175818617970781F0A681B781A20F4E
:102BF000B31F4C93828193810196608171810E9401
:102C000025299383828380E008958FEF0895EF92C2
:102C1000FF920F931F93CF93DF937C01062F10E059
:102C2000B8018CE195E00E94E615D0E0C0E0C01745
:102C3000D10758F4F701EC0FFD1F649170E08CE1AF
:102C400095E00E94E6152196F2CFDF91CF911F917A
:102C50000F91FF90EF900895CF93DF93FC01C28115
:102C6000D38184819581C817D907C9F0A681B7811E
:102C7000A80FB91F2C910196608171810E942529AE
:102C8000C817D90739F095838483822F90E0DF91AC
:102C9000CF9108951582148213821282F6CF8FEF9E
:102CA0009FEFF5CFFC0160817181848195819B014B
:102CB000281B390B82819381820F931F0E94252943
:102CC0000895DC01ED91FC910190F081E02D0994D3
:102CD0008091AA018823B9F08091A901882399F0F5
:102CE0006CE08AED91E00E94071667E083ED91E0C9
:102CF0000E94071667E08CEC91E00E94071661E0E5
:102D00008AE00C94DA0660E08AE00E94DA0667E066
:102D100086EE91E00C9407168F929F92AF92BF922D
:102D2000CF92DF92EF92FF924B015C010E94440729
:102D30006B017C0124E0C21AD108E108F1080E946D
:102D400044076C197D098E099F09681579058A0564
:102D50009B05A8F3FF90EF90DF90CF90BF90AF90CE
:102D60009F908F900895809148048F3F11F42D9883
:102D7000089560E00C94DA06882349F080914804B5
:102D80008F3F11F42D9A089561E00C94DA060C94AB
:102D9000B316CF93DF93EC0181E00E94BC16299A11
:102DA000BE0190E080E00E948C1629980E94B31624
:102DB000DF91CF910C94B3168F929F92AF92BF92F6
:102DC000CF92DF92EF92FF92CF934B015C01219A59
:102DD0008FEF88169806A806B806C1F4219A80E0FD
:102DE00093E20E94C91660EC78E080E090E00E94D7
:102DF0008C1680E392E0CF91FF90EF90DF90CF9020
:102E0000BF90AF909F908F900C94C91680E093E292
:102E10000E94C91660E871E180E090E00E948C1683
:102E2000C0E2C12CD12CE12C90E8F92ED501C401CF
:102E30008C219D21AE21BF21892B8A2B8B2B89F0E0
:102E400080E392E00E94C91660E976E080E090E0BD
:102E50000E948C16F694E794D794C794C15031F72A
:102E6000C8CF80E392E00E94C91660E372E080E080
:102E700090E0EECF2091DA043091DB04C90107968F
:102E800097FD079623E0959587952A95E1F7209180
:102E9000D8043091D904829FA001839F500D929F46
:102EA000500D112470E060E08091F3049091F404DF
:102EB0000C94722AFB0101900020E9F73197AF01D1
:102EC000461B570BDC01ED91FC910280F381E02D54
:102ED00009948F929F92AF92BF920F931F93CF93BB
:102EE000DF93CDB7DEB7A1970FB6F894DEBF0FBE64
:102EF000CDBF19A2423008F44AE08E010F5D1F4F8A
:102F0000842E912CB12CA12CA50194010E9403299F
:102F1000E62FB901CA01EA3004F5E05DD801EE936D
:102F20008D01232B242B252B79F790E080E010973F
:102F300029F0BD0184ED94E00E945A17A1960FB6C6
:102F4000F894DEBF0FBECDBFDF91CF911F910F91DF
:102F5000BF90AF909F908F900895E95CDFCFCF93A3
:102F6000DF93682F70E090E080E04AE00E946917EC
:102F7000EC0160EA71E084ED94E00E945A178C0F36
:102F80009D1FDF91CF9108950F931F93CF93DF93F0
:102F9000EC010E94AB078C0160EA71E0CE010E9457
:102FA0005A17800F911FDF91CF911F910F910895B4
:102FB000CF9324E934E0F90101900020E9F79F0163
:102FC00025593440C0918F0433274C2F50E0BA016B
:102FD00061507109261B370B30938A0420938904B2
:102FE000682F70E06C567B4F88E191E00E94692A5F
:102FF00080911801803219F486E880931801CB5F24
:10300000C0931301EC2FF0E0319620E090E0A92F5F
:10301000B0E0AE5EBE4F4C9124279F5FC917B8F752
:10302000EE5EFE4F20836091130170E06E5F7F4F74
:1030300084E295E00E94E615C0E02C2F30E08091FC
:10304000130190E00196821793075CF02E5E3E4FCD
:10305000F901608170E084E295E00E94E615CF5F9F
:10306000ECCFCF9108950E94642A85ED8093BC0037
:103070008091EC019091ED01A091EE01B091EF01F2
:103080000796A11DB11D23E0B695A7959795879545
:103090002A95D1F72091BC0024FD03C0109235027F
:1030A00008954091EC015091ED016091EE01709115
:1030B000EF01452B462B472B69F30097A105B1057E
:1030C00041F02AE22A95F1F700C00197A109B10960
:1030D000E1CF8091EB010C9478111F93CF93DF9394
:1030E000EC01162F0E94ED28181739F0612FCE0140
:1030F000DF91CF911F910C94F528DF91CF911F9113
:1031000008950C94ED288BE090E00E948118282F00
:1031100030E030930B0120930A018330A1F028F4B2
:10312000813041F0823059F00895843081F085304B
:1031300091F008956AE18AE491E00C9407166AE13F
:1031400082EB91E0FACF6AE188E991E0F6CF6AE19B
:103150008EE791E0F2CF6AE184E691E0EECFCF9383
:10316000DF9390E080E00E948118C82FD0E0D093D8
:103170000901C09308018AE090E00E948118282F7D
:1031800030E03093070120930601219739F4833012
:1031900019F180F48130B1F08230D1F08AE090E012
:1031A0000E94811890E09093070180930601DF91BF
:1031B000CF9108958430A1F0853081F76AE184E6EB
:1031C00091E003C06AE18AE491E00E940716E6CF2D
:1031D0006AE182EB91E0F9CF6AE188E991E0F5CF0D
:1031E0006AE18EE791E0F1CF90E080E00E948118E3
:1031F000282F30E030930501209304018330D9F06B
:1032000028F4813049F0823069F00895853071F1F9
:10321000D0F0873081F108951092A9010E946816BC
:103220000C9483181092A9010E9468166AE180E349
:1032300091E00C9407161092A9010E9468166AE1A9
:1032400086E191E0F6CF6AE18CEF90E00E940716EC
:103250001092A9010E9468166AE186E191E00E943D
:10326000071681E08093A9010C9468166AE182EE4A
:1032700090E00E9407161092A901F6CF4F925F923C
:103280006F927F92AF92BF92CF92DF92EF92FF92B6
:103290000F931F93CF93DF93CDB7DEB768970FB629
:1032A000F894DEBF0FBECDBF7C01FC01D080A280B0
:1032B000C3800481B58016810E949B074090A401C1
:1032C0005090A5016090A6017090A7019B01AC01F0
:1032D000241935094609570929013A0130E14316F5
:1032E00037E253066104710468F06093A40170939F
:1032F000A5018093A6019093A70165E088E690E080
:103300000E94071645E050E06DED70E0C7010E9495
:10331000E028892B29F466E087ED90E00E940716EB
:1033200046E050E061ED70E0C7010E94E028892B83
:1033300019F481E08093AA018091750281110AC07D
:1033400066E082E59CE00E9407160E94F41881E086
:103350008093750245E050E06CEC70E0C7010E947C
:10336000E028892B29F466E086EC90E00E9407169D
:1033700045E050E060EC70E0C7010E94E028892B36
:1033800011F40E94F41840E8D412DAC25FEBA512DF
:10339000DAC288E1C812D7C2B0926702802F90E0EB
:1033A000880F991F909369028093680245E0489FB7
:1033B0009001499F300D11242C5F3F4F43E036951B
:1033C00027954A95E1F730936F0220936E024FE004
:1033D000429FC001439F900D1124839666E470E0E4
:1033E0000E942529615F7F4F6432710510F063E20E
:1033F00070E06093110111E01093740261E081E1CB
:103400000E94DA068091A801811104C00E94F4187C
:103410001093A80168960FB6F894DEBF0FBECDBF1B
:10342000DF91CF911F910F91FF90EF90DF90CF90A0
:10343000BF90AF907F906F905F904F900895153040
:1034400009F4E6C0163031F766E08AE990E00E94A0
:1034500007168091A901882309F420C18091AA014F
:10346000882309F41BC167E083E990E0F6C01A30B5
:1034700009F490C108F046C0183009F414C119309D
:1034800049F690E080E00E94811890E09093090155
:1034900080930801019709F03FC16FE470EB8EE45F
:1034A00091E60E94DC1685E090E090930301809302
:1034B000020180910A0190910B01019686309105DD
:1034C0000CF027C190930B0180930A0160910A01CF
:1034D0008BE090E00E946D1868960FB6F894DEBFFE
:1034E0000FBECDBFDF91CF911F910F91FF90EF9055
:1034F000DF90CF90BF90AF907F906F905F904F9094
:103500000C9483181B3009F484C11C3009F082CF5D
:1035100066E087E890E00E94071665E97AE68EE4A7
:1035200091E62EC2193209F406C258F5163209F492
:10353000E8C140F46FE170EE8EE491E6133209F4D5
:103540001FC268CF173209F4E9C1183209F062CFFF
:1035500062E090E080E068960FB6F894DEBF0FBEA0
:10356000CDBFDF91CF911F910F91FF90EF90DF9032
:10357000CF90BF90AF907F906F905F904F900C94E2
:103580006D181C3209F497C158F41A3209F471C14C
:103590006FE570EA8EE491E61B3209F4F1C13ACF8F
:1035A0001D3209F48DC11E3409F034CF60E08AE089
:1035B00068960FB6F894DEBF0FBECDBFDF91CF91F6
:1035C0001F910F91FF90EF90DF90CF90BF90AF9041
:1035D0007F906F905F904F900C94DA0666E08AEBD4
:1035E00090E00E94071667ED78E28EE491E60E9473
:1035F000DC1680916C02882339F0809110018332AF
:1036000018F48F5F8093100181E08093740202CFE1
:1036100066E084EB90E00E94071667E578EA8EE4A6
:1036200091E60E94DC1680916C02882369F38091F8
:103630001001882349F38150E5CF66E08EEA90E0DF
:103640000E9407168091A90167E08823F1F080911C
:10365000AA018823D1F087EA90E00E9407166896B5
:103660000FB6F894DEBF0FBECDBFDF91CF911F9193
:103670000F91FF90EF90DF90CF90BF90AF907F9031
:103680006F905F904F900C94681680EA90E00E94D3
:10369000071667EB78E48EE491E672C167E378EC95
:1036A0008EE491E66DC166E08DE890E00E94071619
:1036B0006FEA70E58EE491E60E94DC1680910401C9
:1036C0009091050101968630910504F590930501CE
:1036D000809304016091040190E080E00E946D18E5
:1036E00068960FB6F894DEBF0FBECDBFDF91CF91C5
:1036F0001F910F91FF90EF90DF90CF90BF90AF9010
:103700007F906F905F904F900C94F41881E090E060
:10371000DDCF81E090E0D6CE90E080E00E9481187D
:1037200090E09093090180930801029709F072CE0E
:103730008091060190910701019690930701809373
:10374000060120910201309103012817390734F452
:1037500081E090E09093070180930601609106015B
:103760008AE090E00E946D1868960FB6F894DEBF6C
:103770000FBECDBFDF91CF911F910F91FF90EF90C2
:10378000DF90CF90BF90AF907F906F905F904F9001
:103790000C94AF1880910001909101010196863040
:1037A000910594F5909301018093000160910001CF
:1037B00088E290E00E946D1888E290E00E948118F3
:1037C00090E0909301018093000128E1E8E3F1E0AB
:1037D000DE01119601900D922A95E1F7880F991F4D
:1037E000880F991FE1E0F0E0EC0FFD1F8E0F9F1F87
:1037F000FC0160817181828193810E94DC166AEEF6
:1038000075E18EE491E6BCC01092010110920001B6
:10381000CDCF65E77AE88EE491E6B2C061E08AE058
:103820000E94DA068CE00E94B106892B29F060E044
:103830008CE00E94DA0654CF61E08CE00E94DA0648
:103840006AE18DE690E068960FB6F894DEBF0FBE91
:10385000CDBFDF91CF911F910F91FF90EF90DF903F
:10386000CF90BF90AF907F906F905F904F900C94EF
:10387000071680916D0291E0892780936D0288235D
:1038800099F010926C0283E280936B028FE0809338
:103890006A020E949B0760936302709364028093A4
:1038A000650290936602B0CE10926C0210926B0289
:1038B00010926A02A9CE65EC7AE38EE491E660C0CC
:1038C00061E090E080E00E946D1861E08AE090E0A5
:1038D0000E946D1861E08BE090E00E946D1860E03E
:1038E0008EE190E00E946D1860E088E290E00E9416
:1038F0006D1860E08CE890E00E946D180E94F4184A
:1039000033CF8091A901882321F08091AA018111F0
:10391000A6CE6FE870E78EE491E632C08091A901EF
:10392000882321F08091AA01811199CE6FE070EF78
:103930008EE491E625C06FE470EB8EE491E620C042
:1039400020ECD21267CDF1E3CF1264CD61E085E0C7
:103950000E94DA061E3009F461CF08F0E3CD17307B
:1039600009F46BCE08F083CD143009F437CE08F09B
:1039700066CD67E978E68EE491E6133009F04ACD2A
:1039800068960FB6F894DEBF0FBECDBFDF91CF9122
:103990001F910F91FF90EF90DF90CF90BF90AF906D
:1039A0007F906F905F904F900C94DC161F920F9257
:1039B0000FB60F9211242F933F938F939F93AF9342
:1039C000BF938091770290917802A0917902B09193
:1039D0007A023091760223E0230F2D3758F50196B5
:1039E000A11DB11D209376028093770290937802F7
:1039F000A0937902B0937A0280917B0290917C022D
:103A0000A0917D02B0917E020196A11DB11D80930F
:103A10007B0290937C02A0937D02B0937E02BF91C3
:103A2000AF919F918F913F912F910F900FBE0F906B
:103A30001F90189526E8230F0296A11DB11DD2CF25
:103A40001F920F920FB60F9211242F933F934F9313
:103A50005F936F937F938F939F93AF93BF93EF93F6
:103A6000FF93E0910E01F0910F010995FF91EF9105
:103A7000BF91AF919F918F917F916F915F914F9186
:103A80003F912F910F900FBE0F901F9018951F928E
:103A90000F920FB60F9211242F933F934F935F9382
:103AA0006F937F938F939F93AF93BF93EF93FF9306
:103AB000E0910C01F0910D010995FF91EF91BF91FB
:103AC000AF919F918F917F916F915F914F913F91B6
:103AD0002F910F900FBE0F901F9018951F920F926D
:103AE0000FB60F9211242F933F934F935F936F93D1
:103AF0007F938F939F93AF93BF93EF93FF9383E84D
:103B000092E00E944D08FF91EF91BF91AF919F917C
:103B10008F917F916F915F914F913F912F910F9076
:103B20000FBE0F901F9018951F920F920FB60F9215
:103B300011242F938F939F93EF93FF93E091930220
:103B4000F09194028081E0919902F0919A0282FDB5
:103B50001BC0908180919C028F5F8F7320919D028A
:103B6000821741F0E0919C02F0E0ED57FD4F958FF8
:103B700080939C02FF91EF919F918F912F910F90D5
:103B80000FBE0F901F9018958081F4CF1F920F9257
:103B90000FB60F9211242F933F934F935F936F9320
:103BA0007F938F939F93AF93BF93EF93FF938091F6
:103BB000B900887F803609F44AC0F0F5883209F4EC
:103BC000A7C018F5803109F49BC0B8F4882309F424
:103BD000F9C0883009F494C0FF91EF91BF91AF9183
:103BE0009F918F917F916F915F914F913F912F9115
:103BF0000F900FBE0F901F901895883109F488C060
:103C0000803251F78093340214C0803409F49DC08F
:103C100040F48033B9F38833F9F68093340285ECAD
:103C2000B0C0803509F485C0883509F496C0883461
:103C300099F60E943518D0CF883909F48CC038F530
:103C4000883729F050F4883611F0803729F683E060
:103C5000809335021092330257C0883809F47BC034
:103C6000803919F0803809F0B7CF80913302803263
:103C700008F071C0E091330281E08E0F809333022F
:103C80008091BB00F0E0ED5EFD4F80833DC0803B46
:103C900039F0E0F4803A09F479C0883A09F09CCF11
:103CA00084E0809335021092120210921102E0918A
:103CB0005E02F0915F0209958091110281110FC09F
:103CC00081E0809311021092F10109C0803C09F457
:103CD000A6CF883C09F4A3CF883B09F07DCFE091C3
:103CE000120281E08E0F80931202F0E0EF50FE4F3F
:103CF00080818093BB00909112028091110229C0B3
:103D000080915A028093BB0085EC8093BC0064CF05
:103D10009091590280915802981758F5E0915902F4
:103D200081E08E0F80935902F0E0E85CFD4F8081C6
:103D3000E9CFE091590281E08E0F80935902809182
:103D4000BB00F0E0E85CFD4F8083909159028091C8
:103D500058029817C8F285E8D8CFE091590281E05F
:103D60008E0F809359028091BB00F0E0E85CFD4F1C
:103D700080838091370281115CCF81E0809336028D
:103D800084EA8093BC001092350226CF85EC8093A4
:103D9000BC001092350280913302803230F4E09101
:103DA0003302F0E0ED5EFD4F10826091330270E06F
:103DB000E0915C02F0915D0283E192E0099510923E
:103DC00033020ACF1092340234CF1F920F920FB6F3
:103DD0000F9211242F933F934F935F936F937F9391
:103DE0008F939F93AF93BF93EF93FF9381E0809363
:103DF000620260E08DE00E94DA06E1EBF0E0808193
:103E0000887F8083FF91EF91BF91AF919F918F91B8
:103E10007F916F915F914F913F912F910F900FBEC6
:103E20000F901F9018951F920F920FB60F921124AA
:103E30002F933F934F935F936F937F938F939F93B2
:103E4000AF93BF93EF93FF9380E00E94B106019779
:103E5000D9F481E00E94B1060197B1F48091B100DC
:103E600087608093B100FF91EF91BF91AF919F91D7
:103E70008F917F916F915F914F913F912F910F9013
:103E80000FBE0F901F90189580E00E94B106892BFD
:103E900051F781E00E94B106019729F71092620262
:103EA00061E08DE00E94DA068091B100887FD9CF71
:103EB0001F920F920FB60F9211242F933F934F939F
:103EC0005F936F937F938F939F93AF93BF93CF93A2
:103ED000EF93FF93E0913603F0913703C081809117
:103EE0003803C8238091390390913A032091390314
:103EF00030913A032F3F3F4F29F0019690933A03B8
:103F00008093390320913403211115C0C1114BC096
:103F1000813A910558F010924303909346038093A1
:103F2000450381E0809344038093340310923A0365
:103F30001092390338C0213099F4CC23A1F1E091DB
:103F400044032E0F20934403F0E0EC5CFC4F8F3FC2
:103F5000910519F010F08FEF90E0838B82E0E4CFB1
:103F6000223009F047C0E0914403813A910510F4F2
:103F7000E73CA0F1E83C18F081E080934303809196
:103F800045039091460390933C0480933B04E09357
:103F90003A0483E080933403E0913B03F0913C03C7
:103FA000309709F0099580914904882329F081E030
:103FB000C11180E00E94BC16FF91EF91CF91BF919B
:103FC000AF919F918F917F916F915F914F913F91B1
:103FD0002F910F900FBE0F901F901895C111E3CF36
:103FE00091E09E0F90934403F0E0EC5CFC4F838BD8
:103FF00081E09ACF2330B9F6C111D5CF97CFFC011C
:1040000086819781009711F00C94DB29089588E749
:1040100091E09093D5048093D4048091F30490911F
:10402000F404009711F00E94DB2984E295E00E94DD
:10403000FF1F8CE195E00E94FF1F84E195E00C9446
:10404000FF1F0F931F93CF93DF93EC018B017983B5
:1040500068831D821C821B821A82CB010E943F2929
:104060009F838E83A80170E060E0DF91CF911F9164
:104070000F910C94722AEF92FF920F931F93CF939C
:10408000DF93E3E8F2E01382128288EE93E0A0E08F
:10409000B0E084839583A683B78324E531E0318340
:1040A000208325EC30E03587248724EC30E0378707
:1040B000268720EC30E0318B208B21EC30E0338BF5
:1040C000228B22EC30E0358B248B26EC30E0378BD2
:1040D000268B118E128E138E148E28E2E22E23E090
:1040E000F22EF7011382128284839583A683B7830D
:1040F00086E691E0918380830E949B07609324036E
:104100007093250380932603909327030E949B07B7
:1041100060932003709321038093220390932303E1
:1041200060E870E084E195E00E94212060E470E0A6
:104130008CE195E00E94212060E470E084E295E04B
:104140000E9421201FEF10934804E4E3F3E0118262
:1041500001E0048389E290E0938382835098CAE46B
:10416000D4E01CAA0E949B0760932403709325034C
:1041700080932603909327030E949B07609320035C
:1041800070932103809322039093230319861A8648
:104190001B8618861F821E821D8262E080E00E94BC
:1041A000080761E084E00E94080761E084E00E9463
:1041B000DA06E0EBF0E010821092B1008DE9809316
:1041C000B300808182608083E0E7F0E080818260DC
:1041D0008083E8E6F0E0808184608083EDE6F0E0B3
:1041E00080818160808319821A8280ED97E09AAF86
:1041F00089AF88EE93E09CAF8BAF88EC90E09EAFE8
:104200008DAF82E08093900410928A04109289040A
:104210008BE080938F04109291041092920410927C
:1042200093040E949B0760938B0470938C0480938B
:104230008D0490938E04E4EDF4E01382128220E862
:1042400030E03583248380E290E097838683318752
:10425000208793878287168A158614861786168686
:10426000058B048B8FEF9FEF938B828B918B808BD1
:10427000078B108E128E118E88E791E091838083D8
:10428000148E138EF68EE58E10A2178E14A315A32E
:1042900016A317A310A780E89AE1A6E0B0E085ABCB
:1042A00096ABA7ABB0AF80EA96E8A1E0B0E081AFF3
:1042B00092AFA3AFB4AF80E586AF17AEDF91CF91D9
:1042C0001F910F91FF90EF900895789484B58260CC
:1042D00084BD84B5816084BD85B5826085BD85B5AA
:1042E000816085BD80916E00816080936E00109228
:1042F00081008091810082608093810080918100A3
:104300008160809381008091800081608093800033
:104310008091B10084608093B1008091B000816091
:104320008093B00080917A00846080937A008091BD
:104330007A00826080937A0080917A008160809315
:104340007A0080917A00806880937A001092C10090
:1043500010926102109260021092800210927F020D
:104360000E945A1188EA97E090935F0280935E0260
:1043700089EA97E090935D0280935C0268EC70E0BC
:1043800080E090E00E9469078091F3049091F4042A
:10439000892B41F52091DA043091DB04C90107969D
:1043A00097FD0796B3E095958795BA95E1F720912B
:1043B000D8043091D904AC01429FC001439F900DB5
:1043C000529F900D11240E943F299093F4048093F2
:1043D000F304892B39F460EE7BE083E892E00E94DD
:1043E000C417FFCF0E943A172091DA043091DB0402
:1043F0008091D8049091D904B901213231050CF48F
:1044000023C26054710977FF02C06F5F7F4F7595BB
:1044100067958255910997FD019600E410E022E529
:1044200030E04FEE58E0959587950E94241082E089
:104430008093F6048091F1049091F204892B09F4A1
:1044400016C28CE38093F504109261021092600210
:104450001092800210927F020E945A1188EA97E01F
:1044600090935F0280935E0289EA97E090935D02E9
:1044700080935C028091FC0487FD1EC061E00E9475
:10448000080761E08091FC040E94DA0661E070E0B8
:1044900080E090E00E94690760E08091FC040E9447
:1044A000DA066AE070E080E090E00E94690761E06F
:1044B0008091FC040E94DA068091F1049091F2044C
:1044C000892B09F493C22091090530910A05409186
:1044D0000B0550910C0560E074E284EF90E00E94BF
:1044E00003292051310941095109569547953795BE
:1044F00027952093B80064E08BE097E00E940513B5
:104500006091DA04615084ED94E00E94BA1364E093
:1045100087E097E00E9405138091F60460E1813006
:1045200009F064E184ED94E00E94BA1364E083E052
:1045300097E00E9405138FE8809311058091D804BD
:104540009091D9048038910509F067C28091DA040E
:104550009091DB048034910509F06FC28091F604DC
:10456000813009F07DC28FE980931105C2E16AEDC7
:1045700084ED94E00E94BA136C2F84ED94E00E94C5
:10458000BA1361E884ED94E00E94BA1360911105BA
:1045900084ED94E00E94BA1369ED84ED94E00E94EA
:1045A000BA138091F60462E2813009F061EF84ED84
:1045B00094E00E94BA1366E08DEF96E00E94051326
:1045C0008091F1049091F204892B09F44BC220915F
:1045D0000D0530910E0540910F055091100560E0DA
:1045E00074E284EF90E00E940329205131094109CF
:1045F000510956954795379527952093B8000E9405
:104600003A17C1E0C093E804C093E90481E090E068
:104610009093E7048093E6049093E5048093E40488
:104620001092E1041092E0041092E3041092E2046C
:10463000C093EC0463ED7BE084ED94E00E94C4172A
:1046400061EC7BE084ED94E00E94C4176FEA7BE0AC
:1046500084ED94E00E94C4170E941C1461E085E080
:104660000E94080761E086E00E94080760E08AE097
:104670000E94080761E08BE00E94080761E08CE07F
:104680000E94080762E084E10E94080761E08DE073
:104690000E940807E0919302F0919402D2E0D08347
:1046A000E0918F02F09190021082E0919102F091DE
:1046B000920280E1808310929B02E0919702F09138
:1046C000980286E08083E0919502F09196028081C5
:1046D00080618083E0919502F091960280818860EC
:1046E0008083E0919502F0919602808180688083BA
:1046F000E0919502F091960280818F7D808361E048
:1047000085E00E94DA06C09382028FE280938102E4
:104710001092800210927F026FE788E293E00E947D
:10472000EF1188E293E00E941E1283E892E09093DA
:104730004E0480934D04E0919302F0919402D08353
:10474000E0918F02F09190021082E0919102F0913D
:1047500092028FEC808310929B02E0919702F0917D
:10476000980286E28083E0919502F0919602808122
:1047700080618083E0919502F0919602808188604B
:104780008083E0919502F091960280818068808319
:10479000E0919502F091960280818F7D80838CED6F
:1047A00095E0909384048093830488EE93E0909343
:1047B00086048093850488EC90E09093880480932D
:1047C0008704D09390048EE399E1909382048093C0
:1047D000810461E08DE00E94080722E0422E512C06
:1047E00001E010E034E0632E712C43E0A42EB12CE4
:1047F000C1E090E0292E90E0392E80917502811160
:104800000FC068EE73E080E090E00E94690766E008
:1048100082E59CE00E9407160E94F418C09375027E
:10482000E0914F04F0915004E830F10508F026C102
:10483000E45EFB4D0C9439293C2512262826492696
:10484000722687269B26BC266052710977FF02C01C
:104850006F5F7F4F759567958357910997FD019617
:1048600000E210E023E730E04FE057E0DCCD61E00C
:104870008091FA040E94080761E08091FB040E9485
:1048800008078091FA04082E000C990BFC01E257EE
:10489000F34FE491F0E0EE0FFF1FEE59F34F259137
:1048A00034913093020520930105FC01EE55F34F3E
:1048B000E491E09307058091FB04082E000C990B0E
:1048C000FC01E257F34FE491F0E0EE0FFF1FEE59C9
:1048D000F34FA591B491B0930405A0930305FC0197
:1048E000EE55F34FE491E09308058C91E82BEC939F
:1048F0008091EF049091F004892B09F434C0CFB774
:10490000F89480915B02811127C0E8E9FCE0849172
:10491000ECEAFCE09491E82FF0E0EE0FFF1FE85A7C
:10492000F34FA591B491EC91E92321F461E08AE081
:104930000E94DA0661E08AE00E9408078CB5806177
:104940008CBD8CB580648CBD61E08DE00E94080751
:1049500061E08BE00E94080780915B028F5F80938B
:104960005B02CFBF87CD61E08091F8040E94080709
:1049700061E08091F9040E9408078091F804082EF4
:10498000000C990BFC01E257F34FE491F0E0EE0FBD
:10499000FF1FEE59F34F259134913093FE0420937D
:1049A000FD04FC01EE55F34FE491E0930505809181
:1049B000F904082E000C990BFC01E257F34FE49127
:1049C000F0E0EE0FFF1FEE59F34FA591B491B093B5
:1049D0000005A093FF04FC01EE55F34FE491E09332
:1049E00006058C91E095E823EC9344CD8091EF048B
:1049F0009091F004892B31F080911205909113056C
:104A00000E943A0BE0910305F0910405908180919A
:104A100008058095892380836ECD8036910589F4C1
:104A20008091DA049091DB04409739F48091F60488
:104A3000813029F480E180931105C2E098CD8FEA9E
:104A4000FACF80349105C9F78091DA049091DB04A4
:104A5000809799F78091F604813011F480E184CD3C
:104A60008FEC82CDE0910305F09104058081909157
:104A70000805892B8083C3CD109291048091620236
:104A80008823E9F084E295E00E9452161816190670
:104A9000B4F484E295E00E942C166C0180E00E9440
:104AA000B106019739F4F12CE12CF3E1CF16D104D2
:104AB00008F488C1B60184E295E00E94D515809182
:104AC0004D0490914E04DC01ED91FC910084F18540
:104AD000E02D0995892B81F080914D0490914E0431
:104AE000DC01ED91FC910284F385E02D0995BC0178
:104AF00084E195E00E94E615809151049091520462
:104B00008230910509F4B3C108F070C1009709F42F
:104B10007BC1019709F48DC1809162028823D1F194
:104B20008CE195E00E945216181619069CF50E9419
:104B30009B07C0902003D0902103E0902203F090C7
:104B400023036C197D098E099F096A30710581055F
:104B5000910500F18CE195E00E942C166C0180E03B
:104B60000E94B106019739F4F12CE12CB1E2CB1689
:104B7000D1040CF4FEC1B6018CE195E00E94D5157C
:104B80000E949B076093200370932103809322036C
:104B90009093230380914B04882371F00E949B071C
:104BA00060E084E00E94DA0670E060E080914D04ED
:104BB00090914E040E94611680916D02882309F441
:104BC00001C2C0906302D0906402E0906502F09050
:104BD000660280916C028111A7C20E949B076C192A
:104BE0007D098E099F09663971058105910508F4D3
:104BF000E9C1D0916B02DD2309F4CFC167E578EA02
:104C00008EE491E60E94DC16D150D0936B020E9494
:104C10009B07609363027093640280936502909394
:104C20006602CEC1109293041092920480E00E941A
:104C3000D8175092500440924F040E949B076093F3
:104C40008B0470938C0480938D0490938E0416CF04
:104C50000E949B07C0908B04D0908C04E0908D0440
:104C6000F0908E04AB01BC014C195D096E097F09FF
:104C70008091830490918404B0E0A0E04817590724
:104C80006A077B0708F4FACEB0925004A0924F0452
:104C9000F5CE209192048091890490918A0428177E
:104CA000190680F42F5F209392048091930491E081
:104CB000980F909393040E94D817709250046092BA
:104CC0004F04BBCF85E090E09093500480934F0455
:104CD0001092930410929204809191048F5F8093BC
:104CE0009104CCCE0E949B07C0908B04D0908C0482
:104CF000E0908D04F0908E04AB01BC014C195D096D
:104D00006E097F098091870490918804B5CF9091B6
:104D1000910480919004981738F4A6E0B0E0B09325
:104D20005004A0934F0489CFE7E0F0E0F0935004E3
:104D3000E0934F0482CF0E949B07C0908B04D090D9
:104D40008C04E0908D04F0908E04AB01BC014C19F2
:104D50005D096E097F098091850490918604B0E019
:104D6000A0E0481759076A077B0708F487CE10931D
:104D7000500400934F0482CE0E949B07C0908B0486
:104D8000D0908C04E0908D04F0908E04AB01BC01B7
:104D90004C195D096E097F09809185049091860404
:104DA000B0E0A0E0481759076A077B0708F466CE11
:104DB0001092930480E00E94D81710925004109231
:104DC0004F045CCE80904D0490904E04CE14DF04CE
:104DD00009F475CE84E295E00E942C16BC01C40152
:104DE0000E9461162FEFE21AF20AECCF8330910590
:104DF00009F477C061E070E0049709F08DCE84E19A
:104E000095E00E94D515B0C084E195E00E9452164D
:104E1000181619060CF080CE70E060E084E195E091
:104E20000E94BC15809353041093520400935104C4
:104E300073CE84E195E00E94521602970CF46CCE7A
:104E400061E070E084E195E00E94BC158093540419
:104E50008350823228F450925204409251045CCE26
:104E600061E070E084E195E00E94D51555CEC090D8
:104E70005404D12C4601BFEF8B1A9B0A84E195E0C4
:104E80000E945216881699060CF046CED0E0F12CFE
:104E9000E12CB70184E195E00E94BC15D827EFEF23
:104EA000EE1AFE0ACE14DF04A4F7B40184E195E003
:104EB0000E94BC15D817190679F40E949B076093CD
:104EC0002403709325038093260390932703B092C5
:104ED0005204A092510420CE709252046092510468
:104EE0001BCE80915304982F9F77903521F0982FF7
:104EF0009F7B9038C9F48AE4E82E84E0F82E97016D
:104F00002A543440FFEFEF1AFF0A8091540490E0D6
:104F1000019682179307FCF084E195E00E942C161D
:104F2000D7011B968C93EBCF893729F3982F9D7F60
:104F3000983609F38F33F9F28831E9F2982F9F7D83
:104F4000983CC9F26091540470E06E5F7F4F803BE3
:104F500009F055CFD0CFC0937E04E0918104F09149
:104F6000820486E594E0099510925204109251044F
:104F7000D3CDEC14FD040CF003CE80904D04909042
:104F80004E048CE195E00E942C16BC01C4010E94E5
:104F90006116EFEFEE1AFE0AECCFD0916A02DD2324
:104FA00051F067ED78E28EE491E60E94DC16D15074
:104FB000D0936A022CCEFFE0F0931001C0936C02F4
:104FC000C093740280917402882309F491C00E94F6
:104FD0009B07C0907002D0907102E0907202F09036
:104FE00073026C197D098E099F096436710581056C
:104FF000910508F47DC00E949B0760937002709336
:1050000071028093720290937302109274020E9454
:105010003A17C093E804C093E9041093E70400939F
:10502000E6041093E5040093E4041092E104109266
:10503000E0041092E3041092E2046AE47CE084ED60
:1050400094E00E94AB0760916E0270916F0290E055
:1050500080E04AE00E94691765E47CE084ED94E01A
:105060000E94C4176CE37CE084ED94E00E94AB07DF
:105070006091110170E090E080E04AE00E946917C1
:1050800080916D02811177C060E37CE084ED94E053
:105090000E94C41766E07CE084ED94E00E94AB07B8
:1050A000609168027091690290E080E04AE00E949D
:1050B000691760E07CE084ED94E00E94C4176AEF19
:1050C0007BE084ED94E00E94AB076091670244E6C8
:1050D000649FB001112490E080E04AE00E946917CB
:1050E00060EA71E084ED94E00E945A170E941C145B
:1050F0000E949B0761347F418105910548F08BE058
:105100000E94B106019721F460E08BE00E94DA066C
:105110002114310409F471CB0E943908882309F461
:1051200067CB0E94000064CB0E949B076C197D092D
:105130008E099F096C3271408105910508F442CFB8
:10514000D091100180911101D81750F467ED78E2E9
:105150008EE491E60E94DC16DF5FD093100157CDFC
:105160008D1708F02FCF67E578EA8EE491E60E946C
:10517000DC16D150F2CF80916C02811118C0809161
:105180006B02882359F065E27CE084ED94E00E9494
:10519000AB0780916B020E94AF177CCF6AE17CE085
:1051A00084ED94E00E94AB0780916A02F4CF6FE037
:1051B0007CE084ED94E00E94AB0780911001EBCF7E
:1051C000FB01DC0104C08D910590801921F4415050
:1051D0005040C8F7881B990B0895F999FECF92BDEE
:1051E00081BDF89A992780B50895262FF999FECFA9
:1051F0001FBA92BD81BD20BD0FB6F894FA9AF99AF4
:105200000FBE01960895A1E21A2EAA1BBB1BFD0139
:105210000DC0AA1FBB1FEE1FFF1FA217B307E40795
:10522000F50720F0A21BB30BE40BF50B661F771FED
:10523000881F991F1A9469F76095709580959095CD
:105240009B01AC01BD01CF010895AA1BBB1B51E11D
:1052500007C0AA1FBB1FA617B70710F0A61BB70BE6
:10526000881F991F5A95A9F780959095BC01CD018B
:105270000895EE0FFF1F0590F491E02D09940F9310
:105280001F93CF93DF938230910510F482E090E07A
:10529000E0912E05F0912F0530E020E0B0E0A0E095
:1052A000309799F42115310509F44AC0281B390BB0
:1052B00024303105D8F58A819B816115710589F10A
:1052C000FB0193838283FE0111C0408151810281E1
:1052D000138148175907E0F04817590799F41097B8
:1052E00061F012960C93129713961C933296CF018D
:1052F000DF91CF911F910F91089500932E05109388
:105300002F05F4CF2115310551F04217530738F01E
:10531000A901DB019A01BD01DF01F801C1CFEF0155
:10532000F9CF90932F0580932E05CDCFFE01E20F8C
:10533000F31F819391932250310939832883D7CF6A
:1053400020912C0530912D05232B41F4209134011F
:105350003091350130932D0520932C052091320199
:10536000309133012115310541F42DB73EB74091FD
:10537000360150913701241B350BE0912C05F0913B
:105380002D05E217F307A0F42E1B3F0B2817390752
:1053900078F0AC014E5F5F4F2417350748F04E0F91
:1053A0005F1F50932D0540932C05819391939FCFC0
:1053B000F0E0E0E09CCFCF93DF930097E9F0FC01B1
:1053C000329713821282A0912E05B0912F05ED0124
:1053D00030E020E01097A1F420813181820F931FEB
:1053E00020912C0530912D052817390709F061C04F
:1053F000F0932D05E0932C05DF91CF910895EA01FC
:10540000CE17DF07E8F54A815B819E014115510502
:10541000B1F7E901FB83EA8349915991C40FD51F84
:10542000EC17FD0761F4808191810296840F951F2E
:10543000E90199838883828193819B838A83F0E049
:10544000E0E012968D919C9113970097B9F52D91FC
:105450003C911197CD010296820F931F20912C054C
:1054600030912D052817390739F6309751F51092EC
:105470002F0510922E05B0932D05A0932C05BCCFBF
:10548000D383C28340815181840F951FC817D907E8
:1054900061F44E5F5F4F88819981480F591F518396
:1054A00040838A819B81938382832115310509F092
:1054B000B0CFF0932F05E0932E059ECFFD01DC01C8
:1054C000C0CF13821282D7CF81E090E0F8940C9481
:1054D000792AFB01DC0102C001900D92415050403D
:1054E000D8F70895DC0101C06D9341505040E0F7BA
:1054F000089516E0CCE5D6E004C0FE010E943929EB
:0C5500002196CD35D107C9F7F894FFCFF4
:10550C00010001000100010001000100AA07AA0727
:10551C000F0FC80080234232000000000000000082
:10552C00000000000000000000000000000000006F
:10553C0000000000300580007D824E61BD424E614E
:10554C003DC24E61DD224E615DA24E619D624E6197
:10555C00000000006F08CF07FC07BC082D080B08E3
:10556C001F0800000000EF11C211B9158706BB110E
:10557C00A811991100000000780DCF07B915321150
:10558C00830A87061D10F50F11100510851087066C
:10559C003E0B6315F3093C0A3E0F210FA90E4A0E70
:0455AC000D0A0000E4
:00000001FF
